:0400000002002B329D
:01000B0032C2
:0100130032BA
:01001B0032B2
:030023000200AB2D
:0300840002002651
:0500260012010380FE41
:07008700752200752300C281
:0C008E0000759850740F5589F5F074202F
:0E009A0045F0F589758DFC758780D28ED2AC4D
:0300A800D2AF22B2
:0C00AB00C0E0C0D075D01010980280009A
:0500B700109902801EFB
:0600BC00E522B52304C299
:0300C200008015A6
:0500C500D200AA220593
:0A00CA0022EA2424F8869974F82530
:0600D4002250037522001A
:0500DA00D0D0D0E0329F
:0A00DF00AA82E5232424F8A602E516
:0600E9002304FABA08002E
:0400EF0040027A0051
:0800F300EAB52204C2B480F852
:0700FB008A23200002D299C4
:0101020022DA
:0C010300D2B4C2B3D2B5D2B312008774DC
:0A010F0089C0E07407C0E07480C0EE
:0E011900E01201A3158115811581C2B4C2B395
:05012700E4F52CF52DAC
:0A012C00C3E52C9405E52D648094D2
:0A01360080501420B20A052CE4B535
:060140002CEA052D80E60B
:07014600E4F52CF52D80DF2C
:0C014D008590821200DFC2B5E4F52CF5AD
:010159002D78
:0A015A00C3E52C9405E52D648094A4
:0A01640080501430B20A052CE4B5F7
:06016E002CEA052D80E6DD
:07017400E4F52CF52D80DFFE
:04017B00D2B580A8D1
:0E0789004D616E75616C205054522C20465705
:0E079700312E30312C20342F32342F323031BD
:0E07A500360D0A4572696B2042616967617208
:0E07B3002C204765726D616E790D0A0D0A00EB
:06005A00E4787FF6D8FDFA
:080038007900E94400601B7A25
:05004000009007CC78E0
:030045000075A0A3
:0A00480000E493F2A308B8000205DB
:08005200A0D9F4DAF275A0FF59
:080060007800E84400600A7911
:030068000075A080
:06006B0000E4F309D8FCDB
:080071007800E84400600C79FE
:0B00790000900000E4F0A3D8FCD9FACE
:06017F00C0098581091290
:0501850000DFD009229B
:08018A0085823D85833E85F06E
:050192003FE4F53AF521
:040197003BF53C8573
:03019B0008409089
:05019E00017F02026375
:0601A300C009858109E599
:0701A9000924FBF540E4F519
:0401B0003AF53BF5EC
:0701B4003CE50924FBF8867D
:0601BB003D08863E0886A7
:0501C1003F90017F12D8
:0501C6000263D00922D4
:0701CB00AA82C030C031C060
:0601D2003274E2C0E0748B
:0601D80001C0E0C02EC0D2
:0401DE002F8A8222C0
:0A01E2001581158115810538E4B57B
:0401EC003802053997
:0101F00022EC
:0E01F100AA8274302AFA24C6500A74072AFA29
:0601FF0030010343022061
:050205008A820201CB1A
:0E020A00E582FAC4540FF582C0021201F1D051
:0902180002740F5AF5820201F193
:0602210085820AAB33AC3C
:0402270034AD35AE0F
:04022B0036AF37753E
:02022F000B20A2
:0E023100EF2FFFEE235401FA4207EB2BFBECFC
:0C023F0033FCED33FDEE33FEC3EF950AF7
:0A024B004008EFC3950AFF430301CA
:06025500D50BD98B338CA0
:04025B00348D358E1B
:04025F00368F37227D
:0702630085822E85832F85A3
:03026A003A3085A2
:03026D003B31859D
:040270003C32E4F543
:0302740038F53921
:05027700AA3DAB3EAC06
:0C027C003F8A828B838CF0120769FD74AE
:09028800012AF53DE43BF53E8C32
:080291003FEDFA700302074A79
:05029900BA25028003FC
:03029E0002074212
:0502A100C202C203C20D
:0402A60004C205C2C7
:0402AA0006C207C2BF
:0402AE0008C2097504
:0802B20041007542007DFFAE22
:0402BA003DAF3EAB6B
:0102BE003F00
:0E02BF008E828F838BF0120769FAA3AE82AF96
:0602CD00838E3D8F3E8B85
:0B02D3003FBA25078A821201CB8099F8
:0502DE008A04BC3000A1
:0D02E300402A8A04EC24C64023BDFF13E529
:0B02F0004275F00AA4FCEA24D02CF5B3
:0702FB004270C1D20380BD77
:0D030200ED75F00AA4FCEA24D02CFD80B0BB
:0A030F00BA2E07BDFFAA7D0080A6EC
:050319008A04BC610034
:0D031E00400E8A04EC248540075302DFD214
:03032B000180024C
:02032E00C2010A
:05033000BA2002805517
:05033500BA2B02804B11
:05033A00BA2D02804114
:05033F00BA4202804BF0
:05034400BA43028050E5
:06034900BA44030204F4B3
:06034F00BA460302050A94
:06035500BA49030204F4A2
:05035B00BA4C028034E1
:06036000BA4F030204FB8A
:06036600BA500302048BF3
:05036C00BA5302804CB1
:06037100BA55030205006D
:06037700BA58030205055F
:03037D0002050E68
:05038000D2020202BFE1
:05038500D2040202BFDA
:05038A00D2050202BFD4
:05038F00D2070202BFCD
:05039400D2080202BFC7
:0803990030070AE54014F88862
:0503A100408602800F00
:0A03A600E54024FEF88840860308B5
:0503B0008604188B0219
:0803B5008A821201CB02051738
:0A03BD00E54024FDF888408603089F
:0A03C700860408860618188B338C94
:0403D100348E3585AC
:0603D500338285348385AC
:0C03DB0035F0C005120751AB82AC83D096
:0603E70005BDFF028B05BD
:0A03ED0020022CC3EB95425026E5D8
:0603F70042C39BF542AC7D
:0103FD0042BD
:0C03FE008C061C8C42EE6014758220C03E
:0E040A0003C004C0051201CBD005D004D003FE
:0204180080E47E
:02041A008C4212
:02041C008D044D
:07041E0085338285348385DC
:0C04250035F0120769FDFA602F8C051CF1
:0E043100C374808DF063F08095F050208A82B5
:0C043F00C003C0041201CBD004D003ADF8
:04044B0033AE34AFE9
:06044F00350DBD00010E99
:050455008D338E348F91
:03045A003580C129
:06045D0020020302051756
:09046300C3EB95424003020517AA
:07046C00E542C39BF542AC21
:010473004246
:0B0474008C051C8C42ED700302051586
:0C047F00758220C0041201CBD00480E97B
:0A048B00E54024FDF88840860508CE
:0A049500860608860718188D338EBE
:04049F00348F35E57C
:0A04A30035FD247F50047A438014D5
:0904AD00ED249F50047A50800BED
:0904B600ED24BF50047A498002D4
:0204BF007A5869
:0E04C1008A82C0021201CB75823A1201CB75FD
:0E04CF0082301201CB7582781201CBD002BAB6
:0404DD004902800B45
:0504E100BA5002800684
:0604E60085348212020AB7
:0804EC0085338212020A80230D
:0704F400D20675410A801CCD
:0504FB007541088017A7
:0505000075410A8012A4
:05050500754110800D9E
:04050A00D209800989
:07050E008A821201CB80027A
:020515008C4216
:0905170030095AE54024FCF88883
:0C05200040860408860508860608860749
:08052C001818188C338D348E71
:04053400358F367554
:0305380033C17557
:03053B003407750D
:02053E00358006
:040540008533448536
:03054400344585B6
:0505470035467401259A
:07054C0044FFE43545FCAD5E
:04055300468F338C10
:04055700348D358525
:06055B0044828545838502
:0A05610046F0120769FCFA7003026D
:02056B00027715
:07056D008A821201CB80CC51
:07057400E54170030202776C
:04057B0075431D3077
:07057F00072BE54014F8888A
:0A05860040E6FD3395E0FEFFFC8D1A
:04059000338E348FE3
:04059400358C36204C
:0A059800065EAC337D007E007F009C
:0505A2008C338D348E46
:0505A700358F36804C89
:0905AC0030081FE54024FCF8882A
:0C05B500408604088605088606088607B4
:0805C1001818188C338D348EDC
:0505C900358F36802A89
:0A05CE00E54024FEF888408604088A
:0C05D800860518ED3395E0FEFF8C338D96
:0405E400348E358F8D
:0505E8003620060CACFA
:0805ED0033AD347E007F008E67
:0305F500358F3609
:0A05F800300622E53630E71BC3E4AD
:090602009533FCE49534FDE49508
:07060B0035FEE49536FF8C7B
:04061200338D348E62
:05061600358F36800263
:02061B00C20615
:06061D00D20AA8437C0094
:0A062300753700854182C004C00055
:0B062D00120221D000D004200A0DE5CD
:0A06380037C4FDE6FE4DF6188843B6
:02064200800234
:02064400A637D7
:080646000C8C03B20AE53345F8
:04064E0034453545B5
:080652003670CE88438C03E5ED
:06065A004270037542012D
:0A066000200324200221EB04FCAD6E
:01066A00424D
:0E066B00C3EC9D5015758220C003C004C0056D
:0C0679001201CBD005D004D0031D80E698
:020685008D42A4
:0C06870030060E75822DC0031201CBD08E
:05069300031542802365
:0C069800EB602030040E75822BC00312B2
:0806A40001CBD0031542800FC9
:0C06AC0030050C758220C0031201CBD079
:0306B800031542E5
:0506BB00200224AC4206
:0B06C0008C051C8C42C3EB9D502B30BE
:0606CB0003047D308002F3
:0206D1007D208A
:0E06D3008D82C003C0041201CBD004D003807E
:0106E100DE3A
:0A06E200C3EB95425008E542C39BAC
:0406EC00F54280074C
:0506F0007542008002CC
:0206F5008C4235
:0206F700A84316
:0A06F9008B041BEC6026B20A200AF5
:0B0703000A08E6C4540FFC8C37800786
:07070E008604740F5CF5374F
:0C071500853782C003C0001201F1D00043
:04072100D00380D4AD
:060725002002030202772E
:02072B00AB42DF
:09072D008B041BEC70030202773F
:0C073600758220C0031201CBD00380EBC1
:080742008A821201CB0202774A
:07074A008538828539832206
:0B07C1003C4E4F20464C4F41543E0080
:04075100AA82AB834A
:080755001207696003A380F89C
:0C075D00C3E5829AF582E5839BF58322B8
:03002B0075814696
:0A002E00120785E582600302002638
:0E07690020F71430F6148883A88220F507E6E6
:06077700A8837583002237
:03077D00E280F720
:03078000E49322DD
:02078300E02272
:040785007582002257
:00000001FF
